:030000000219FDE5
:03000B000200AA46
:03002B0002018748
:03005B000203415C
:0300730002032E57
:1000800002030406080C10182030406080040608A3
:100090000C10182030406080A0C00003070F1F0D17
:1000A0000D04050D050305030302C2AF306308C24A
:1000B0006385798AD2AF32C0D0C0E0206221E525C5
:1000C0006016E473E525F4C3334009758A00D263F2
:1000D000F57901D6F58AD262D0E0D0D0D2AF32C362
:1000E000E526334009758A00D263F57901F0F58A77
:1000F000C262E526F4602F30682520720DD0E0D072
:10010000D0C295C293C297D2AF32C295C293C29762
:10011000206F0C2065097412D5E0FDE57B4290D07C
:10012000E0D0D0D2AF32758A00D263757900C28D2B
:10013000D262211F01C4306805206502D29501C436
:10014000306805206502D29701C430680520650239
:10015000D29301C4C29430680A2065077412D5E0B6
:10016000FDD29501C4C29630680A2065077412D585
:10017000E0FDD29701C4C29230680A20650774126C
:10018000D5E0FDD29301C4C2AFC2AD53E6EFC0D0FB
:10019000C0E0D2D3D2AFE57A6009E5776005757724
:1001A0000041DB757701C2CEE52A600720744F1548
:1001B0002A21FE7800790020742EE580307E01F43B
:1001C00030E50278FF53DACF207E0343DA20307E19
:1001D0000343DA10C2D8C271E580307E01F430E505
:1001E0000279FFC3E89970CB306103752A18207437
:1001F00003752A18885CD270E86003755F0020746C
:100200000DE52B6004152B410E43DA01C2D8207096
:1002100002417DA85C206102C2702074367982B7E9
:100220000431C3E894F0400374F0F8E8C4540F2894
:10023000F87984B703024153C313C31387212008FD
:1002400002C313200A06C3C898F8415328F8500384
:1002500074FFF88822E52D54066022206B1FE536D6
:10026000C333C333F8E564C313C313F9C395224002
:10027000028922E82522F52250037522FF7882B6F2
:100280000459852224A824C3E52495614002A8616D
:10029000C3E895634002A8638825E566700241CEF5
:1002A000C3E8AA669A5003E8FAE4F9EAC333FBE527
:1002B00068F45B29400D2567F8E567600215674023
:1002C0000B41CE0AC3E5679A5002056778FF88267E
:1002D000C26FC3E52694F84002D26F20CF0AD0E067
:1002E000D0D043E610D2AD32C2CF053AE57A6009EC
:1002F000E578600575780061247578017801E52A54
:100300006005307402152AC3E55C94014005755FF1
:10031000006124756000756900E55F2401F55F5098
:1003200003755FFFD0E0D0D043E610D2AD32C2AF4C
:1003300053E67F7592FA7593FFC260759104D2AF50
:1003400032C2AF53E6EFC2ADC0D0C0E0C0F0D2D3EE
:10035000D2AFA8FBA9FCE57A6007C3E913F9E8135B
:10036000F8C2D830710261B353DACF207E0343DA8A
:1003700010307E0343DA20D271E580307E01F42014
:10038000E502618A88278928A1E053DACF207E031D
:1003900043DA20307E0343DA10C2D8C271307402CF
:1003A000A1CC7800E580307E01F430E502A1CC8854
:1003B0005CA1B453DACF207E0343DA20307E0343BE
:1003C000DA10C271206102818C53DACF207E0343A0
:1003D000DA10307E0343DA20C2D8D27188578958A8
:1003E000C3E89555F8E99556F97B007E087A00C375
:1003F000E8948CE994005005755B00817E88217833
:10040000A2E6A8216055C3E894C8E994005008E426
:10041000D2E4FB7A0A8159C3E89468E99401500850
:10042000E4D2E3FB7A0F8159C3E894D0E9940250F7
:1004300008E4D2E2FB7A1E8159C3E894A0E994054E
:100440005008E4D2E1FB7A3C8159C3E89498E994DE
:10045000085008E4D2E0FB7A787E00C3E89559FCA6
:10046000E9955AFD30E70AECF42401FCEDF4340080
:0E047000FD755B00C3EC9AED9E5003755B01B9
:10047E008859895A8557558558567802A1B4C3E8CC
:10048E009527F8E99528F9307C02A198307B02A1D6
:10049E0098307A02A19120750281AFE9FDE8FC81C6
:1004AE00CEE9C313F9E813F8307902A191E9C31329
:1004BE00F9E813F8307802A191E9C313FDE813FCB3
:1004CE0020612CC3EC941CED9402400281E5ED708A
:1004DE001EC3EC94C850180529E52970021529C3CE
:1004EE00E529940A5002A1CC755C00D270A1CCE52E
:1004FE0029600215297888E6F97400207F0878961D
:10050E00B90302789EE624FAFEE43400FFC3EC9EA3
:10051E00FCED9FFD9208B90310A208500720760942
:10052E00D276A137307602C276A2085016B9030DE4
:10053E00ECF42401FCEDF43400FD02055178007951
:10054E0000A198B90315EC33FCED33FDC3EC940A0E
:10055E00FCED9400FD50047C007D00C3EC94FFED97
:10056E009400400678FF7900A198EC8572F0A4C53E
:10057E00F0A2F733F8790040030205B478FF790052
:10058E000205B4E9C313F9E813F8307C0EE96002F2
:10059E0078FFC3E81338F8E43400F9C3E894FFE9B0
:1005AE009400400278FF885CD270206102A1CC7466
:1005BE001FF4552F4BF52FC274EB7002D274752AAF
:1005CE0018307403752A0A306102A1E020740353B7
:1005DE00DAFE207403752B06D0F0D0E0D0D0D2AD69
:1005EE0043E6103279010206107903020610790AE9
:1005FE00020610791E020610796402061079C802EE
:10060E0006107817E4D5E0FDD8FAD9F6227A147BD5
:10061E00780206377A107B8C0206377A0D7BB4028D
:10062E0006377A0B7BC8020637E573D5E0012279CF
:10063E0002E4C296D5E0FDD297D5E0FDC297D5E093
:10064E00FDD296D5E0FDE920E002D29530E002D24F
:10065E0093E573D5E0FDE920E002C29530E002C2D9
:10066E00937496D5E0FDD9C9EAF8D5E0FDD8FBDB49
:10067E00B8C29622C37C007D0075F00005F0EA3307
:10068E00FAEB33FB50F6EB13FBEA13FAC3E9FFE880
:10069E00FEE89AF8E99BF95004EFF9EEF8B3EC3363
:1006AE00FCED33FDD5F0DFEDF9ECF822E889F08AA8
:1006BE0020D2D4F8A9F07B0030F70B7BFFF4240195
:1006CE00F8E9F43400F9E88520F0A4ADF0F8E985F6
:1006DE0020F0A4AFF0FEED2EF974003FFA7C04C3B7
:1006EE00EA13FAE913F9E813F8DCF48BF030F70AA1
:1006FE00E8F42401F8E9F43400F9E889F0C2D4F8FA
:10070E00A9F0227882B6040302076CC3E55C94015B
:10071E004003020736852224E4F544F545F546F5F7
:10072E0047F548C26E02076C7882E6FCD26EE5226F
:10073E00F523783879C7AA40AB41C3EB13FBEA1314
:10074E00FAEC146013C3EB13FBEA13FAEC14146007
:10075E0007C3EB13FBEA13FAD1828844894522C3FF
:10076E00E5449523F8E5459400F9500CC3E89480D0
:10077E00E994FF401602079DC3E8947FE994005068
:10078E000302079D787F790002079D788079FF88A4
:10079E0049894A22E5492546F8E54A3547F9854A09
:1007AE0020E4300701F43548FA30E709C3EA94F043
:1007BE0040150207DBC3EA940F50030207DB78FFF4
:1007CE0079FF7A0F0207DB780079007AF0C3E5240F
:1007DE009561500AC374019524500B0207F9E54A3E
:1007EE0020E70E0207F9E54A30E706884689478A70
:1007FE00482278A5E6FAC3E54933F8E54A33F912FB
:10080E0006BAE930E70BC3E89480E994FF40130180
:10081E0034C3E8947FE9940050020134787F790064
:10082E000134788079FFE820E715C3E52398F84076
:10083E0009C3E89401400302085B780102085BE8F3
:10084E00F424012523F8400302085B78FF884B222D
:10085E0078A6E6FAA847A9481206BAE930E70CC30B
:0F086E00E89401E994FF4016020890C3E894FF54
:10087D00E99400500302089078FF790002089078FF
:10088D000179FFE920E715C3E54B98F84009C3E866
:10089D00940140030208B778010208B7E8F4240177
:1008AD00254BF840030208B778FF88242278FF20F3
:1008BD00692879A1E76023E541601F74FF8541F048
:1008CD00848539F0306A0375F005A4F8C5F060022F
:1008DD0078FFC3E895645002A864886322C3E5409D
:1008ED0094C8E5419400E56350031401FB046002D4
:1008FD00F563220209032275E890227883E6FF3022
:10090D00EDF9A8BDA9BE0570C3E5709408405275F8
:10091D007000E9FA79A0E76044EA7007E571601BA1
:10092D0002093CC3E895716010E5715006600C1426
:10093D000209480460F9020948E571F571C3947222
:10094D00401B7561C0C394044013756180C394044A
:10095D00400B756140C39404400375610075BB087D
:10096D0022E5612410500274FFF5617982B704020B
:10097D002195C3A861E524985002A824C3E8956386
:10098D004002A86388258826E570B4070375BB105F
:10099D0022743279A787F0A4C5F0A2F733F8C3E823
:1009AD0095614002A861882288248825882688645C
:1009BD00227540007541F022C2AF75C820A8CCA9A0
:1009CD00CDAA3A30CF010A75C824D2AFC3EA13FAC3
:1009DD00E913F9E813F8AB3BAC3C883B893CC3E821
:1009ED009BF8E99C20690A547FF930660241E44185
:1009FD003EAD3D8A3DF9EA9D547FFA600678FF7958
:100A0D00FF4123AE3EAF3F8B3E8C3FA83BA93CC37D
:100A1D00E89EF8E99FF9C3E54113FBE54013FAE8B9
:100A2D002AF540E93BF54150067540FF7541FF4100
:100A3D008BAA40AB41AC40AD417E047F02C3EB9429
:100A4D0004400D1E1FC3EB94084005206A021E1FB3
:100A5D00C3ED13FDEC13FCDEF7C3EA9CFAEB9DFB33
:100A6D00EF6009C3E913F9E813F8DFF7EA28FAEBA9
:100A7D0039FB8A408B4150067BFF8B408B41C3EB8A
:100A8D0094025002D2663069047F0341B67892E633
:100A9D00FFC3E537948240110FC3E53794A04001A1
:100AAD000FC3EF940640027F057E02E541C4540F4B
:100ABD00F9E541C454F0F8E540C4540F28F8C3E8F3
:100ACD009EFAE99400FB4009C3EA9402EB940050AE
:100ADD00047A02E4FB6130AA40AB41EBC4FEEAC4E8
:100AED00540F4EFCC3EA9CFAEB9400FBC3E813C30E
:100AFD0013F8EA28FAEB3400FB8A408B41C3EB94E0
:100B0D00024002C2667802EBC4FE7B00EAC4540FB9
:100B1D004EFAC3EA98FA4005C3940250027A02785D
:100B2D0092E6FF3060026130855192855293D2601A
:100B3D0043E680C3E49AF8E49BF9C3E833F8E9335C
:100B4D00F930660261C3E8FAE9FBD3E913FDE81356
:100B5D00FC88518952C3EF94036038EF20E00DE813
:100B6D002CF8E93DF9ECFAEDFB020B8CE828F8E9DD
:100B7D0039F9C3E82402F8E93400F97AFE7BFFC3A2
:100B8D00EF9403400E8A538B54884D894E8C4F8DB4
:100B9D005061F7885389548A4D8B4E8C4F8D503050
:100BAD0069127553F07554FF754FF07550FF7551FF
:100BBD00F07552FF61F7E8FAD3E813FC8851C3EFE3
:100BCD0094036020EF20E007E82CF8ECFA61E3E8ED
:100BDD00282402F87AFEC3EF940340088A53884D07
:100BED008C4F61F788538A4D8C4FE568C3335002A3
:100BFD00646BF5683060028101753402D26043E6A2
:100C0D0080E52D5406602DA840A941C3E913F9E8EC
:100C1D0013F8306904E92440F9C2AF53E67F7591AA
:100C2D0000C3E498F594E499F595759104D2604369
:100C3D00E680D2AF22D264754300752000306C037C
:100C4D00752040020C61D264754300752040306CF4
:100C5D000375200078017901206620E52D5406608A
:0E0C6D0002C2647914E541C313700104F8C398
:100C7B00941440027814306904781B791BC3E83351
:100C8B00F8C3E933F9206010E543600C306903D5F4
:100C9B003404D26DA11791090543E59B5440B5204F
:100CAB0002A10130690908C3E8994001188190201D
:100CBB00640A08C3E899400281618190C264C2AFA3
:100CCB0053E67F7591003066127594007595F0753B
:100CDB009104D26043E680D2AF8161E5417EFFC3D0
:100CEB00334009C3334005C3334001FEC3E49E7553
:100CFB009400F59581DAC3E533940150028161309C
:100D0B0064028161D802A1158190C26DC2AF53E616
:100D1B007F759100855394855495759104854D92FB
:100D2B00854E93D26043E680D2AFE52D5406600822
:100D3B00206A020533020D53306D0D206C0A2064BE
:100D4B00071581158102161A22780030640278018A
:100D5B00E53775F007A4F9E5F028F5F0E9A2F013F3
:100D6B00A2F113A2F213F537C394785003753778B9
:100D7B00C3E53795384008D265C295C293C2973008
:100D8B006002A18A854F92855093D26043E6802200
:100D9B00207D16C2AF754202C296D294306202D247
:100DAB0093D2AF759F11020F8BC2AF754202C296E1
:100DBB00D292306202D295D2AF759F11020F8B3057
:100DCB007243207D20C2AF754203900165757B4055
:100DDB00C293C292306204D297A1E8D296D2AF7579
:100DEB009F13020F8BC2AF754203900165757B4059
:100DFB00C295C294306204D297C108D296D2AF7515
:100E0B009F10020F8B207D17C2AF754203900140DC
:100E1B00C293306202D297D2AF759F13020F8BC26F
:100E2B00AF754203900140C295306202D297D2AFA8
:100E3B00759F10020F8B207D16C2AF754204C294B2
:100E4B00D292306202D297D2AF759F10020F8BC233
:100E5B00AF754204C292D294306202D297D2AF7570
:100E6B009F13020F8B307243207D20C2AF7542055A
:100E7B00900154757B10C297C296306204D295C113
:100E8B008ED294D2AF759F11020F8BC2AF754205F4
:100E9B00900176757B04C297C296306204D293C1DF
:100EAB00AED292D2AF759F11020F8B207D17C2AFBE
:100EBB00754205900136C297306202D295D2AF755A
:100ECB009F11020F8BC2AF75420590014AC297303A
:100EDB0062EBD293D2AF759F11020F8B207D16C29E
:100EEB00AF754206C292D296306202D295D2AF75DE
:100EFB009F13020F8BC2AF754206C294D29630621B
:100F0B0002D293D2AF759F10020F8B307244207DAB
:100F1B0020C2AF754201900176757B04C295C294D5
:100F2B00306204D293E134D292D2AF759F10020F8C
:100F3B008BC2AF754201900154757B10C293C29264
:100F4B00306205D295020F55D294D2AF759F130222
:100F5B000F8B207D17C2AF75420190014AC29530AD
:100F6B006202D293D2AF759F10020F8BC2AF754244
:100F7B0001900136C293306202D295D2AF759F13A6
:100F8B00C26522900134757B00C295C293C297C291
:100F9B0094C292C296C262227880760908760908BA
:100FAB0076040876FF0876030876FF08760A08763B
:100FBB0003087601087601788C76010876FF0876AF
:100FCB00FF0876FF0876FF0876FF0876030876FFA2
:100FDB000876FF0876FF0876250876D0087628086D
:100FEB0076500876040876FF0876020876000876B5
:100FFB007A0876FF087601087601087600087603F2
:10100B00087600227887E6FFC272BF0302D272789D
:10101B0088E6C394036008C27DE630E102D27DC24C
:10102B007E7889E630E102D27EC3EF9402600875C8
:10103B008E01D273021047758E00C273227880E640
:10104B00149000809378A5F67881E6149000809335
:10105B0078A6F67886E61490008D9378A7F67886B6
:0E106B00E6F539C394025003753902789CE60D
:101079007538FFB402037538A0B403037538827854
:10108900A3E61490009A93F566120F8E22227896A1
:10109900E6FA7897E6FB7888E6B40305C3EB940E85
:1010A900FB307F047A007BFFC3EB9AFCC394825028
:1010B900027C827572000572EC8572F0A4C3E5F0BA
:1010C900947D40F222D27F11971206011206017A0D
:1010D900007B007C101205F7E55C2AFA74003BFBE3
:1010E900DCF37C04C3EB13FBEA13FADCF7FEC27FE3
:1010F900119722757C00757D00E5EF20E6037520C8
:10110900000520903FFFE520146006901FFF146042
:10111900009304600375EF1653D9BF7581C043FF6F
:10112900801205F275EF0643B203E5B3240220E706
:101139000DF521E5E320E0068521B343E301120F14
:101149008E7580FF75A40075F1B275D4DF759001B5
:1011590075A5FC75F2FE75D50175A60175E24112FA
:101169000F8EE4F8F6D8FD756801120FA3121673F5
:1011790078988673753001C2AF12060B12061B12DE
:101189000601120622120601120629120601C2AF31
:10119900757C00757D0078FA79FA308507D9FBD816
:1011A900F7021C00110F1148119611977898867350
:1011B900120F8E75A90075B680757A00758810753D
:1011C900890275C82475910475D84075A82275B827
:1011D9000275E690759B80759D0075D10E75BCC032
:1011E90075BB0875BA1175E8801205F2D2AF1209FC
:1011F9000075360053DACF207E0343DA20307E03B0
:1012090043DA1043DA01C2D8C27112060BD2617BEC
:10121900037A0CE55B70077A0CDB0302119712065F
:1012290001207003021197C270E55CC3940240E18A
:10123900E52F541F855E5DF55EB55DD5DAD5C261D2
:1012490053DACF207E0343DA20307E0343DA10C21B
:10125900D8C27178A2E67008D274E52F54E0F52F50
:10126900C275752900120606307409C3E529940A66
:101279004002D2751205F778023074027800C3E58E
:101289005C9840F0C2AF12061B12061B12061BD255
:10129900AF12060B754C007888E6B403026193120D
:1012A90005F7788CE6C394015003021393E530C324
:1012B90094015003021393757CA5757DF120743553
:1012C900C3E55C94FF5003021393C2AF120630D2F8
:1012D900AF120606C3E55C940150EFC2AF12061BBC
:1012E9001205FC12061BD2AF120606C3E55C94FF79
:1012F90040E902182B7F02D27F1197120606C2AF6E
:10130900C27F1197AE5CC3E55C947FD2AF50026196
:10131900A31205F2C2AF120630D2AFDFDA11CEC383
:10132900EE7897F612060B1217AE7F0AD27F119745
:10133900120606C2AFC27F1197AE5CC3E55C947F0B
:10134900D2AF50E61205F2C2AF12061B1205FC120B
:10135900061BD2AFDFD611CEEE24037896F6F879C4
:1013690097E7C394824003985006E824827897F659
:1013790012060B1216C11217DD1206061197C3E5E4
:101389005C94FF500241C002182B757C00757D00EA
:10139900C3E55C954C4003855C4C120606780179DF
:1013A90088E7B403027805C3E55C98400241A0C20E
:1013B900AF120630120630120630D2AF12060B7584
:1013C9003000E4F531F5320531E531F4703F05328D
:1013D900789AE67819146012783214600D787D14C1
:1013E900600878FA146003753200C3E53298401D2D
:1013F900120F8E1205F2153275310078998673C273
:10140900AF120630D2AF789886731206061205FC21
:10141900E52A700530740221977801207402780654
:10142900C3E55C9840A17888E6C39403600312067B
:1014390006E52A7003021197C2AF120F8EE4F52256
:10144900F523F524F525F526F567D2AF7885E6C3AA
:1014590033F565E4F544F545F546F547F548F57086
:0F146900F52CF52DF53775700875BB101205F2CF
:1014780012090430EDFDA8BDA9BEE97001F8887114
:1014880012090875700875BB10110FC2AF7561FF9E
:1014980012099E852261852262852263D2AF752258
:1014A80001752401752501752601856069756A0134
:1014B80075B69075A903757A017888E6B40307C2F2
:1014C8007D307602D27DD268D269753300120EE77C
:1014D800120F161209BE1209C51209BE1209C51249
:1014E80009BE120C53120711120D54120D9B12094A
:1014F800C5120C42306E0312076D2066031208BA3B
:101508003066031208EA120D54120DCA1209C512E8
:101518000C53306E031207A2120D54120E41120919
:10152800C5120C42306E03120800120D54120E70D0
:101538001209C5120C53306E0312085E120D5412B4
:101548000EE71209C5120904120C42120D54120FAB
:10155800161209081209C53069328564618564620A
:10156800856069756A0179187A0CC3E53399400F6B
:10157800C269D26A8A35856461856463021594C339
:10158800E55C940140030214EA021622306A252021
:101598006C22E535147006C26AD26B81EAF535C350
:1015A800E55C940140030214EA7888E6C39403607A
:1015B8000302162275360078FA79A4E760027803E8
:1015C800C3E55F985054307404E52A604D7888E686
:1015D800B40317207D05207607A1F2307602A1F228
:1015E800206C07D26C856461A12978F0306C058580
:1015F80064617820C3E54198500281EA306C1BC2CF
:101608006CC27D307602D27DD26A753512856461EE
:1016180081EA0536E55C6002C125753600C2AF1265
:101628000F8E7887E6FE7602110F7887EEF6E4F5DE
:1016380022F523F524F525F526F565752C00752D7D
:101648000075A90075B680757A00D2AF1206061229
:101658000F8E78A4E66006D295D297D2933074099B
:10166800C3E53694044002219761CB901A0D782087
:10167800121703E520B4550CA3121703E520B4AAEA
:10168800030216A1757CA5757DF1120FA31216C170
:10169800757C00757D000216C0901A0378807B0A5D
:1016A800121703A308DBF9901A0F788C7B1912170D
:1016B80003A308DBF9901A2822C2AF1217461217A3
:1016C80023901A00740E121708A37409121708A39E
:1016D8007415121708901A0378807B0A121707A34B
:1016E80008DBF9901A0F788C7B19121707A308DB0F
:1016F800F9121759121737901A2822E493F622E69E
:10170800438F01538FFDFFC3E583941C400122EFF3
:10171800857CB7857DB7F0538FFE22438F02438FB8
:1017280001857CB7857DB7901A0DF0538FFC229008
:101738001A0D7455F108901A0E74AAF108227A301D
:1017480079D07820901A40F103E520F709A3DAF759
:10175800227A3079D0901A40E7F10809A3DAF92201
:10176800AB74A875BB01027980BB02027981BB0307
:10177800027982BB04027984BB05027986BB060222
:101788007992BB07027987BB080279A3BB09027962
:101798009CBB0A027988BB0B027989E8F7227C0591
:1017A80012060BDCFB22C2AF12061B12062212061F
:1017B800291206301205FC12061B120622120629EF
:1017C8001206301205FC12061B12062212062912F6
:1017D8000630D2AF22C2AF120630120629120622F4
:1017E80012061B1205FC12063012062912062212D6
:1017F800061B1205FC1206301206291206221206D2
:101808001BD2AF22AE74AF75C2AF12061B12061BF5
:1018180012061B1205FCDEF21206301205FCDFF878
:10182800D2AF221217AE1217A61217A67574017539
:101838007501757600110C7C05AD5C12060BC3EDC5
:10184800955C70F5C3E55C9401400AC3E55C94FFC0
:10185800403702186E1217681216C11217AEC2AFBF
:0F18680075EF161217A6DCD10576C3E57694034B
:10187700500280C21217A60575E5741490009F9355
:10188700F808C3E57598500280A91217A61217A683
:101897000574C3E574940C50028095120FA31216B9
:0918A700C1C2AF75EF161217A6BD
:0319FD000210FCD9
:101A00000E0915090904FF03FF0A03010155AA0184
:101A1000FFFFFFFFFF03FFFFFF25D0285004FF0259
:091A2000007AFF0101000300FF40
:101A4000234656544C6962656532304150726F23AB
:101A500023424C48454C492346333930232020202B
:101A60002020202020202020202020202020202076
:101C0000C2AFC2D353D9BF7581C043B20343FF8073
:101C1000752438752503B1DC7529A5752AF175E29F
:101C20004043F12053A4DF75D4FFD2857DFA7803B9
:101C300079E67C10752200752300901DE97B0675FE
:101C400024987525013085028145208508D8FBD967
:101C5000F9DCF781B7308508D8FBD9F9DCF781B713
:101C6000B19CE493A3C39A6004DDC381B7DBDBB10D
:101C70008E6002812E7B08E493FAA3B16FDBF87AC1
:101C800030B16F752200752300B18EEAFCEBFDC305
:101C9000ED94FE400EB18E8A278B28ED30E0048A49
:101CA000828B83B18E7AC270D8C3ED94FE601950D6
:101CB000CEBD002BEC600F7520007521FF7529004B
:101CC000752A000200008100A827A9280809D80465
:101CD000D90281DCB192EA89AAF281CE0D81A3C337
:101CE000ED94035053EDA2E092007AC5C3E58294CF
:101CF00000E583941C508A200010438F02438F011B
:101D00008529B7852AB7F0300029A827A92808090E
:101D1000438F01538FFDD804D902A133C3E58394C7
:101D20001C4003A3A11689AAE28529B7852AB7F02A
:101D3000A3A116538FFC817F7AC1BD030CE493A34A
:101D4000FAB153DCF8B14B817F8181AA22AB23B178
:101D50006FEBFAEA6222752608C3E52313F523E543
:101D60002213F52250066323A0632201D526EAB18F
:101D7000DCB1DC75260AEAF4200102D285300102CA
:101D8000C285B1DCC3134002C201D526EB22B19259
:101D9000EAFB208502A192308502A197752608AE44
:101DA00024AF25C3EF13FFEE13FEB1E0B1DCC3EAAD
:101DB000133085024480FA30E703632201C3E52330
:101DC00013F523E52213F52250066323A0632201B5
:101DD000D526D9E52265236523F52222AE24AF2539
:101DE0000E0FDEFEDFFCD20122424C48656C6934E6
:071DF000373164F390060196
:00000001FF
